:040000009031002813
:1000080070082000A10080312100911E5F28200087
:10001800911E5F2823009D1C1B281D121908200013
:10002800EF0023001D162200B80A0319B90A23009D
:100038001D1D28289D139D172200B80A0319B90A07
:10004800230019082000EF00230019082000EF0002
:100058006F080D3A031D46280130A9000030AA0098
:1000680021009112A03020004D07860000304E3D3F
:10007800870081014D08CF004E08D000CD01CE0188
:10008800EF015F28A0304D07860000304E3D870005
:100098006F0881004D08CF004E08D000CD0A031923
:1000A800CE0A00304E02031D5B2850304D02031C5F
:0E00B8005F28CD01CE0120002108F0000900D4
:1000C60023009E1868280000632825003D082300A9
:0400D6009A00080084
:1000DA00240014197A281F301605F1007108003A15
:0E00EA00031D7A280130F0007B28F001080089
:0A00F80071088A00700882000800F9
:100102002000911125003708240091002000510899
:100112002500B800200052082500B900200053082D
:100122002500BA00200054082500BB002400141D3D
:10013200C028200051085204530454040319BF2854
:100142002500380839043A043B04031DB82822006C
:10015200620886006308870004308100413160082C
:10016200F0006108F1007C200130F000002901302C
:100172002500B8020030B93BBA3BBB3B97282000B0
:1001820051082500B800200052082500B9002000BF
:1001920053082500BA00200054082500BB002000A7
:1001A2009119F82851085204530454040319F728EA
:1001B2002500380839043A043B04031DF0282200C4
:1001C20062088600630887000430810041316008BC
:1001D200F0006108F1007C200130F00000290130BC
:1001E2002500B8020030B93BBA3BBB3BD028240003
:1001F200161BFD28F001002916150230F000080038
:060202002400161508009F
:10020800FB14FB1F0E29FF30F300F200F100F00091
:08021800FA0DF20CFF300800A2
:10022000200051082500B900200052082500BA001E
:10023000200053082500BB00200054082500BC0006
:10024000B701B8013808123C031D282937088E3C35
:10025000031C34296D20700803192F293429250027
:10026000B70A0319B80A2229250012303802031DE3
:100270003B298F303702031C40297B30F0006C296A
:10028000240016142400161C6B2920005108520467
:100290005304540403196A29250039083A043B041D
:1002A0003C04031D6329220062088600630887005E
:1002B0000530810041316008F0006108F1007C20C8
:1002C0000130F0006C2901302500B9020030BA3B42
:0A02D000BB3BBC3B4229F0010800D3
:0E02DA00F201F101F001F801F301003008001B
:1002E8007B15FB1F7E290130F300F201F101F001BB
:0802F800FA0DF20CFF300800C2
:08030000FA1FF213003008009F
:10030800A0017208031D99297108F2007008F10014
:10031800F001A0157208031D99297108F200F10176
:10032800A011201672080319A7292008F302031D3B
:10033800031CAB290310F21BAF29F00DF10DF20DD0
:10034800F30B9F29AB290130FC006D21B229023043
:0E035800FC007421B2290430FC008021080052
:10036600102125003408B700812070082500B6004A
:100376000030F100FF307106031DC329FF307006FF
:10038600031DC7292400951325003508B7008120D1
:1003960070082500B600012125003608F000080087
:1003A6007C18092AFC18DA297C19282AD329A001E5
:1003B6007208031DFA297108F2007008F100780826
:1003C600F000F801A0157208031DFA297108F20061
:1003D6007008F100F001A01120167208031DFA2919
:1003E6007108F200F101A015720803191C2A2008F1
:1003F600F302031D031C202A0310F21B092AF80D21
:10040600F00DF10DF20DF30B002A202A7B1B701C58
:10041600242AF81F242AF00A0319F10A0319F20AFA
:10042600031D242AF20CF10CF00CF30A0319282AF6
:10043600242A0130FC006D212B2A0230FC00742195
:100446002B2A0430FC0080212B2A0830FC000421D2
:04045600000008009A
:10045A002000F801F9011030FC00710DF80DF90DBA
:10046A007408F8027508031C750FF9020318442A68
:10047A007408F80775080318750FF9070310F00DCB
:08048A00F10DFC0B322A080001
:10049200200072087606A000F801F90173087702BD
:1004A200031C6B2A7708FD007308F7007D08F30030
:1004B2007608FD007208F6007D08F2007508FD005E
:1004C2007108F5007D08F1007408FD007008F40061
:1004D2007D08F00077080319E42A7208FA00F2177F
:1004E200F61777087302F70003199E2A083077027D
:1004F200031C942AF7007408F9007508F4007608C2
:10050200F500F60108307702031C942AF7007408FC
:10051200F9007508F400F50108307702031C942AEB
:100522007A08F200E42A770803199E2A0310F60CCF
:10053200F50CF40CF90CF70B972AA01FAB2AF9095A
:10054200F409F509F609F90A0319F40A0319F50A77
:100552000319F60A7908F80774080318740FF007EC
:1005620075080318750FF10776080318760FF2075E
:10057200A01BC42A031CD42AF20CF10CF00CF80CB8
:10058200F30FD42AE02A0318D82AF809F009F1094E
:10059200F209F80A0319F00A0319F10A0319F20A17
:1005A2008030FA06DC2A0130FC00D321E62A023030
:1005B200FC00D321E62A0430FC008421E62A08301C
:0E05C200FC000421E62A0030FC0000000800C6
:1005D000F03025003205F000F01570147008B300FB
:1005E000220066082500B40004307004B500B32171
:1005F00070082200E800E9010330FD00FD0BFE2A2F
:1006000066082500B400FB303305B500B32170083F
:100610002200E800E9010330FD00FD0B0D2B250051
:100620003208F000F035F035F035F035F030F005F7
:10063000F01570147008B300220066082500B4009D
:1006400004307004B500B32170082200E800E9010D
:100650000330FD00FD0B2A2B66082500B400FB309B
:100660003305B500B32170082200E800E90103302A
:08067000FD00FD0B392B080011
:06067800FB15FF30080035
:10067E007B14FB1F4A2BF201FA1FFF30F200F10030
:0A068E00F000FA0DF20CFF30080036
:0A06980020008030F6064922080019
:1006A2002000FB01730803198D2B7208FA00F21760
:1006B2008E30F302F31F902BF309F30A0830730212
:1006C200031C732BF300F10D7208F100F2010830E4
:1006D2007302031C732BF300F10DF1017308031D68
:1006E20003107B2B730803197B2B0310F20CF10C04
:1006F200F30B762B7B1B711C852B031C852BF10ABC
:100702000319F20AF21B9C2BFA1F9F2BF209F10923
:10071200F10A0319F20A9F2BF201F1019F2B7B14BC
:10072200FB1FA22BF201FA1FA22BFF30F200F100F5
:10073200FA0DF20CA22B0130FC00A42B0030FC00BD
:10074200A42BFF30FC00FC080319A82B3F237108DF
:08075200F0007208F10008003C
:10075A007408003A031DC62B7508003A031DC62B00
:10076A007608003A031DC62B7708003A031DC62BEC
:10077A00FF30F000FF30F1007F30F200FF30F3006D
:10078A00602C200077080319542C73080319572C7E
:10079A00720876068039FA00F217F617A001720875
:1007AA00F8007108FC007008FD007408FD02750865
:1007BA00031C750FFC027608031C760FF802F80179
:1007CA00FC01FD01031CF02B0310F20CF10CF00CE0
:1007DA00F80C0130A0007708F302031CFA2B7E30D4
:1007EA002007F30703185A2CFF2B7E302007F30744
:1007FA00031C5D2C1830FA07FD0DFC0DF80DF00DE9
:10080A00F10DF20DA00D7408F0027508031C750FA6
:10081A00F1027608031C760FF202760DA004201C62
:10082A00182C7D14232C7408F00775080318750F0B
:10083A00F10776080318760AF2077D10FA031F30CB
:10084A007A05031D012C7B1B7D1C4A2C0310F00D1D
:10085A00F10DF20DA00D7408F0027508031C750F56
:10086A00F1027608031C760FF202760D2004013994
:10087A00FD070318FC0A0319F80A031D4A2CF80C91
:10088A00FC0CFD0CF30A03195A2CFA1FF81378080A
:10089A00F2007C08F1007D08F00000305F2C013086
:1008AA003C235F2C02306D215F2C043004215F2C25
:0808BA00083074210000080061
:1008C20025002E0884002F0885000008F00070081B
:1008D20003197E2C2E0884002F0885000008F000E2
:1008E2002C0886002D08870070088100AC0A0319C5
:1008F200AD0AAE0A0319AF0A612C2C0886002D0836
:06090200870081010800DE
:100908002300EF0105306F020318962C6F082500AD
:100918002E07860000302F3D8700203081002300FD
:10092800EF0A862C6F0825002E07860000302F3D21
:10093800870081012300EF036F0825002E07B00010
:1009480000302F3DB1000A30F400F5012C08F0000A
:100958002D08F1002D227808F0007908F1003030D8
:10096800F0072500300886003108870070088100EC
:100978000A30F400F5012C08F0002D08F1002D22B2
:1009880070082500AC007108AD0000307106031D29
:10099800CF2C00307006031DD22CD52C2300EF037A
:0409A800A02C080077
:1009AC002500AE012C0884002D08850000082300CA
:1009BC00EF006F08003A0319F32C6F082500BD00F7
:1009CC0063202500AE0A2E082C07840000302D3D34
:0C09DC00850000082300EF00DF2C08005D
:1009E8002000FA017308031D7A147708031DFA140E
:1009F8007A0803193F2D033A03190A2D7A18072D8F
:100A0800F61F3D2D3B2DF21F3B2D3D2D72088039E1
:100A1800FA00F21376088039F6137A060319182DAE
:100A28007A0803193B2D3D2D7708730203191F2DF2
:100A3800031C332D372D760872020319262D031C4B
:100A4800332D372D7508710203192D2D031C332DF5
:100A5800372D7408700203193F2D0318372DFA0833
:100A680003193D2D3B2DFA0803193B2D3D2D031489
:0E0A780008000310080003140315080008000E
:100A86002500AE01AF012C0884002D088500000862
:100A9600003A0319682D80302F06F000803070026E
:100AA600031D572D14302E020318682D2C088400C0
:100AB6002D0885000008B200E8222500AC0A0319BB
:0C0AC600AD0AAE0A0319AF0A462D080065
:100AD20020007008F8007108F000F101F201F30142
:100AE200FB01FC019630F300FA01F01F7E2DF8099C
:100AF200F009F80A0319F00AFA177008F1007808E9
:0A0B0200F000F801F2018421080060
:100B0C0025002E08F4002F08F5002C08F2002D0803
:100B1C00F3003008F0003108F1000130B002003071
:100B2C00B13B700871040319AC2D7408840075086E
:100B3C008500720886007308870000088100F20A9D
:100B4C000319F30AF40A0319F50A8F2D2C08F00087
:060B5C002D08F100080065
:100B62002000FB017308031D77080319072E720882
:100B72007606FA007708F3077E30031CC42DF302D1
:100B820003180A2EC72DF302031C0D2E7208F8005B
:100B92007108FC007008FD00F817F6170310F20147
:100BA200F101F0011830A0007D1CE12D7408F0075E
:100BB20075080318750FF10776080318760FF20708
:100BC200F20CF10CF00CF80CFC0CFD0C0310A00B59
:100BD200D52DF21BF12DF80DF00DF10DF20DF303F1
:100BE2007B1B701C032EF81F032EF00A0319F10A57
:100BF2000319F20A031D032EF20CF10CF00CF30A96
:100C020003190A2EFA1FF21300300F2E01306D2144
:100C12000F2E023004210F2E043074210000080030
:100C2200F03025002C05F000F01570082300EF00CD
:100C3200220066082500B40004307004B500B32118
:100C420070082200E800E9010630FD00FD0B272EA6
:100C5200000066082500B400FB3023006F05250064
:100C6200B500B32170082200E800E9010630FD005A
:100C7200FD0B392E000025002D080319732E2C08B8
:100C8200F000F035F035F035F035F030F005F015C4
:100C920070082300EF00220066082500B40004302B
:100CA2007004B500B32170082200E800E9010000D9
:100CB20000000000000066082500B400FB3023009D
:100CC2006F052500B500B32170082200E800E90194
:100CD2000D30FC00FB30FD00FD0B6D2EFC0B6D2E6C
:060CE20000000000080004
:100CE8000D302500BD0063200A302500BD006320BB
:020CF8000800F2
:100CFA002300640884006508850000086606031D51
:100D0A008B2E6408F0006508F1009D2E6408F0003F
:100D1A006508F100E40A0319E50A700884007108FD
:100D2A0085000008F0007008031D7D2EF001F10116
:020D3A000800AF
:100D3C00CF2E20000C11220064082500AC002200EC
:100D4C0065082500AD00E730AE009830AF00612497
:100D5C00DC2E20000C15220064082500AC002200BB
:100D6C0065082500AD001130AE009930AF0061244C
:100D7C00DC2E20000C11220064082500AC0022009F
:100D8C0065082500AD00FC30AE009830AF00612442
:100D9C00DC2E23006408013A03199F2E6408023AE2
:100DAC000319AF2E6408033A0319BF2E0B30FB0056
:100DBC002630FC005D30FD00FD0BE22EFC0BE22E1C
:100DCC00FB0BE22E00000000200011109601970191
:100DDC0018140230FB000430FC00BA30FD00FD0B8F
:100DEC00F52EFC0BF52EFB0BF52E0000181017083A
:100DFC002300E600E501200016082300E50700307B
:100E0C00E63D2000111C0E2F2200EA0A0319EB0A02
:100E1C00230065082500AC00230066082500AD0002
:100E2C00A030AE000130AF0084240E3022006407E5
:100E3C002500AC0000302200653D2500AD00A0303F
:100E4C00AE000130AF000530B0000030B100862597
:100E5C00220064082500AC00220065082500AD00C6
:100E6C00D62474266B2FC0302500AC000130AD00A9
:100E7C001126782F003020005606031D472F023014
:100E8C005506031D4F2F94302500AC000130AD00EA
:100E9C00112620000C11782F200000305606031D5F
:100EAC00592F02305506031D622FD4302500AC009B
:100EBC000130AD001126682F94302500AC000130B4
:100ECC00AD00112620000C11782F23006408013A84
:100EDC000319392F6408023A0319402F6408033AA6
:100EEC000319522F4130FC00EE30FD00FD0B7C2F1E
:100EFC00FC0B7C2F0000220064082500AC002200B3
:100F0C0065082500AD0043251030FB003930FC008E
:100F1C000D30FD00FD0B902FFC0B902FFB0B902F39
:100F2C000000000023006508F0006608F1000800CE
:100F3C00230064088400650885000008F000700830
:100F4C000319B42F64088400650885000008250087
:0E0F5C00BD006320E40A0319E50A9E2F080079
:100F6A00230064088400650885000008F000700802
:100F7A000319CC2F64088400650885000008250041
:100F8A00B200E8222300E40A0319E50AB52F080093
:100F9A002300E601E701640884006508850000086B
:100FAA00F1007108003A0319F52F80306706F00046
:100FBA0080307002031DE32F143066020318F52FE8
:100FCA00640884006508850000082500B200E8224C
:100FDA002300E40A0319E50AE60A0319E70AD02FEF
:020FEA000800FD
:100FEC00230064089100920195131513151413082E
:040FFC00F0000800F9
:1010000023006A08003C031C0A280730EB0000306C
:10101000EC001D286A08163C031813281730ED0051
:101020000030EE0019286A08013EED00EE010030A4
:10103000EE3D6D08EB006E08EC006B082500A60085
:1010400023006C082500A700A001A101F401F5010F
:10105000F601F70123006408F0006508F100660856
:10106000F2006708F3008031F4248831013003185E
:101070000030F000700803194F282300680886002C
:10108000690887002D308100E80A0319E90A003059
:10109000E4060030E5068030E6060030E70623006F
:1010A0006408F4006508F5006608F6006708F700B4
:1010B000F001F101F201F3018031F42488310130B3
:1010C00003180030F00070080319A4280030F40061
:1010D0000030F5000030F6007F30F7002300640890
:1010E000F0006508F1006608F2006708F30080313F
:1010F000F4248831013003180030F000700803191F
:10110000A42823006408F0006508F1006608F200D6
:101110006708F3000030F4000030F5002030F600DE
:101120008230F7008031B125883170082300E40057
:101130007108E5007208E6007308E7000130250039
:10114000A0020030A13B66280030F4000030F5001A
:101150002030F6008230F70023006408F0006508B4
:10116000F1006608F2006708F3008031F42488314A
:101170000130031C0030F00070080319E128003032
:10118000F4000030F5002030F6008230F700230034
:101190006408F0006508F1006608F2006708F300D3
:1011A0008031AD23883170082300E4007108E50028
:1011B0007208E6007308E7002500A00A0319A10AD7
:1011C000A42825002008A6072108A73D0130A20079
:1011D0000030A3000030A8000030A9000030AA00B1
:1011E0007F30AB0080302306F0008030270670028D
:1011F000031DFC282608220203181E290030F400D3
:101200000030F5002030F6008230F7002808F000AA
:101210002908F1002A08F2002B08F3008031AD23E1
:10122000883170082500A8007108A9007208AA007A
:101230007308AB00A20A0319A30AF2280030F400D5
:101240000030F5000030F6008030F7002808F0008C
:101250002908F1002A08F2002B08F3008031AD23A1
:10126000883123006408F4006508F5006608F6007C
:101270006708F70080314922883170082300E400B4
:101280007108E5007208E6007308E7000030F4001A
:101290000030F5002030F6008230F7008031F42471
:1012A00088310130031C0030F000700803196529F3
:1012B00000302300E4000030E5000030E6007F301D
:1012C000E7002500A00A0319A10A250080302106A5
:1012D000F00080307002031D6F29003020020318D7
:1012E000B42923006808860069088700303081002F
:1012F000E80A0319E90A68088600690887002E30A1
:101300008100E80A0319E90A803025002706F00069
:1013100080307002031D8E290030260203189429A4
:101320002608A0022708A13BFF30A200FF30A3003F
:1013300080302106F000803023067002031DA229B0
:10134000220820020318B4292300680886006908CF
:10135000870030308100E80A0319E90A01302500CE
:10136000A2020030A33B9829A201A30180302306EA
:10137000F000803027067002031DC02926082202D3
:101380000318392A23006408F0006508F100660894
:10139000F2006708F300803151238831700825007E
:1013A000A4007108A5003030F0072300680886000B
:1013B0006908870070088100E80A0319E90A250016
:1013C00023082106031DE62920082206031DF22911
:1013D000230068088600690887002E308100E80A2B
:1013E0000319E90A25002408F0002508F1008031DE
:1013F0006925883170082500A8007108A9007208C5
:10140000AA007308AB007008F4007108F5007208B8
:10141000F6007308F70023006408F0006508F10087
:101420006608F2006708F30080314C2388317008A9
:101430002300E4007108E5007208E6007308E70085
:101440000030F4000030F5002030F6008230F70064
:101450008031B125883170082300E4007108E5006F
:101460007208E6007308E7002500A20A0319A30A20
:10147000B6292300680886006908870081010800F2
:1014800023006408F2006508F3007208F000730896
:10149000F100F20A0319F30A70088400710885004C
:1014A00000080319542A452A64087202F0006508EE
:0E14B000733BF1000130F0020030F13B080008
:1014BE0020007008F8007108F000F101F201F3014C
:1014CE00FB01FC019630F300FA017008F100780878
:0E14DE00F000F801F20180318421883108000D
:1014EC0023006808F000E80370080319AB2A6408AD
:1014FC008400650885000008003A0319942A6608E0
:10150C008400670885000008F10064088400650801
:10151C00850000087106031D942AA42A640884001F
:10152C00650885000008F0006608840067088500DF
:10153C000008F002F1010030F13BAD2AE40A031976
:10154C00E50AE60A0319E70A762AF001F101080018
:10155C0001302500AC000130AD00803111268831FE
:10156C0002302500AC000130AD00803111268831ED
:02157C00080065
:10157E00A4302300E4009930E50080319E278831A5
:10158E0080302500AC000130AD008031112688314D
:10159E008F302300E4009930E5008031CD2788316B
:1015AE0020000C160B30FB002630FC005D30FD00D9
:1015BE00FD0BDF2AFC0BDF2AFB0BDF2A00000000ED
:0215CE00080013
:1015D0004D2B80302500AC000130AD00803111264C
:1015E00088317A302300E4009930E5008031B52756
:1015F000883180302500AC000130AD0080311126EB
:1016000088316E2BC0302500AC000130AD00803138
:10161000112688317A302300E4009930E5008031CA
:10162000B5278831C0302500AC000130AD008031D5
:10163000112688316E2B94302500AC000130AD00AE
:101640008031112688317A302300E4009930E5009A
:101650008031B527883194302500AC000130AD00D1
:101660008031112688316E2BD4302500AC0001303A
:10167000AD008031112688317A302300E4009930A2
:10168000E5008031B5278831D4302500AC00013029
:10169000AD008031112688316E2B003022006F069C
:1016A000031D542B01306E060319E92A00306F0622
:1016B000031D5C2B02306E060319022B00306F06EF
:1016C000031D642B03306E0603191B2B00306F06BD
:0E16D000031D6C2B04306E060319342B08002A
:1016DE00003023006106031D762B003060060319CF
:1016EE00B02B600884006108850000080319B02B38
:1016FE006208E4006308E50040227008E800600814
:10170E00E4006108E5006208E6006308E70076225F
:10171E0000307106031D952B00307006031D9C2BA7
:10172E006008F0006108F100B22B01306007E400A0
:10173E000030613DE5006208840063088500000802
:10174E00E60080317D2688317008E0007108E100E6
:08175E006F2BF001F1010800FE
:10176600FB302300E4009930E50080319E27883164
:1017760080302500AC000130AD0080311126883163
:101786007E302300E4009830E5008031CD27883193
:1017960020000C120B30FB002630FC005D30FD00F3
:1017A600FD0BD32BFC0BD32BFB0BD32B0000000024
:0217B600080029
:1017B8002200EA01EB0102302000D5000030D600FB
:1017C8000C160C110B30FB002630FC005D30FD00C0
:1017D800FD0BEC2BFC0BEC2BFB0BEC2B00000000A7
:1017E80080302500AC000130AD00803111268831F1
:1017F80093302300E4009830E5008031CD2788310C
:101808000630FB001330FC00AD30FD00FD0B0A2C48
:10181800FC0B0A2CFB0B0A2C000000000130E40032
:1018280080319E26883170082000DB007108DC00BA
:101838005F227008E7007108E8007208E900730881
:10184800EA0002302300E40080319E2688317008C7
:101858002000D7007108D8000A305C02031D362C1E
:1018680000305B02031C4B2C22006B08003C031D5C
:101878003F2C6A08003C031C4B2C00302000580603
:10188800031D482C0030570603194B2C912CAE220F
:10189800C0302500AC000130AD0080311126883100
:1018A8002A302300E4009830E5008031CD278831C4
:1018B80094302500AC000130AD008031112688310C
:1018C8003F302300E4009830E5008031CD2788318F
:1018D800D4302500AC000130AD00803111268831AC
:1018E80054302300E4009830E5008031CD2788315A
:1018F800CF30E4008F30E50080319E278831663094
:10190800FB007630FC00C130FD00FD0B892CFC0B80
:10191800892CFB0B892C0100362D20005708F0007C
:101928005808F1005F227008EB007108EC0072089B
:10193800ED007308EE007008F4007108F5007208F5
:10194800F6007308F7006708F0006808F1006908F6
:10195800F2006A08F3008031AD2388317008E30093
:101968007108E4007208E5007308E60070082300B7
:10197800E4007108E5007208E6007308E700A0308B
:10198800E8000130E9000430EA0000202E30E400CD
:101998009A30E50080319E278831A0302500AC00C0
:1019A8000130AD008031D6248831803174268831E9
:1019B80020006308F0006408F1006508F20066087A
:1019C800F3006308F4006408F5006508F60066088B
:1019D800F7008031B12588310030F4000030F5007F
:1019E8000030F6007F30F70080314C2388317008D2
:1019F800E3007108E4007208E5007308E600700867
:101A08002300E4007108E5007208E6007308E700A7
:101A1800A030E8000130E9000430EA000020B730C7
:101A2800E4009930E50080319E278831A0302500F8
:101A3800AC000130AD008031D62488318031742665
:101A4800883120000C111530FB004B30FC00BE30F3
:101A5800FD00FD0B2D2DFC0B2D2DFB0B2D2D00005E
:061A6800D501D6010800C3
:101A6E00200098019817181398121812981118152B
:101A7E00181499131913991219129910191022008A
:061A8E00EA01EB01080073
:101A94004E302200E6001030FB003930FC000D30DF
:101AA400FD00FD0B532DFC0B532DFB0B532D0000A0
:101AB400000030302500AC00AD01803111268831A2
:101AC4008230FC00DD30FD00FD0B662DFC0B662D25
:101AD4000000000030302500AC00AD01803111263B
:101AE40088313430FC00F130FD00FD0B772DFC0B08
:101AF400772D0000000030302500AC00AD018031AE
:101B0400112688313430FC00F130FD00FD0B882DA6
:101B1400FC0B882D0000000020302500AC00AD0136
:101B24008031112688313430FC00F130FD00FD0B8A
:101B3400992DFC0B992D0000000028302500AC00E5
:101B44000130AD008031112688313430FC00F13091
:101B5400FD00FD0BAB2DFC0BAB2D0000000008308D
:101B64002500AC000130AD008031112688313430BD
:101B7400FC00F130FD00FD0BBD2DFC0BBD2D000064
:101B8400000001302500AC000130AD008031112689
:101B940088310230FB000430FC00BA30FD00FD0B3C
:101BA400D12DFC0BD12DFB0BD12D000006302500CF
:101BB400AC000130AD008031112688313430FC0096
:101BC400F130FD00FD0BE42DFC0BE42D00000000C2
:101BD4000C302500AC000130AD0080311126883175
:101BE4003430FC00F130FD00FD0BF62DFC0BF62D1E
:061BF400000000000800E3
:101BFA00F101F20180307206F00080307002031D9C
:101C0A00082E503071020318152EA0307107860075
:101C1A000030723D87008101F10A0319F20AFF2D93
:101C2A002000CF01D001F101F201230019082000A0
:0E1C3A00EF00EF01A901AA0121009116080098
:101C480012001E00F003031D242EF103031D242E91
:021C5800080082
:101C5A0022006E082300E000E10123006008E4008E
:101C6A008031F627883170082200EF007008003AA8
:101C7A00031D402E662E8030F0008030230061065E
:101C8A007002031D4A2E6008FE3C03184D2E662E74
:101C9A0022006F082500BD008031632088310D3095
:101CAA00FC00FB30FD00FD0B582EFC0B582E0000EB
:101CBA000000E00A0319E10A22006F08003A031D36
:041CCA00322E0800AE
:101CCE0063302200A8000030A900BD30AA00023007
:101CDE00AB00FF30BE00FF30BF000030C000003050
:101CEE00C100FF30C200FF30C3000030C40000301E
:101CFE00C500FF30BA00FF30BB000030BC00003022
:101D0E00BD0023009E1690309D0021008D140D11F4
:101D1E002000911E962E23001908F0008F2E080029
:101D2E006D302200D8000030D9000030DA000030CB
:101D3E00DB001030DC000130DD000030DE00003052
:101D4E00DF00FF30B000FF30B1000030B2000030D5
:101D5E00B300FF30B400FF30B500FF30B600FF30E7
:101D6E00B7008130AC000030AD00B730AE000230AD
:101D7E00AF000130A4000130A5000030A6000030F5
:101D8E00A70024001413941321008D140D1638305F
:061D9E002400950008007E
:101DA40022001D179D169D171E1423009F1020004E
:081DB4009E0121000D1508003D
:101DBC00FF3021008D00FF308C0020008C012300AF
:101DCC008C0121000C110C1220000C160C1123009C
:101DDC008D0124008C168D0121008D140D128D1295
:101DEC000D150D170D148D15220091019201930103
:041DFC009401080046
:1020000098313A2290318831DE26903120000C162A
:102010000C1120302200E4000230E50023009F155F
:10202000CF309B009C011E1588316726903102300D
:10203000FB000430FC00BA30FD00FD0B1D28FC0B3A
:102040001D28FB0B1D2800008831D226903102305C
:10205000FB000430FC00BA30FD00FD0B2D28FC0B0A
:102060002D28FB0B2D2800002000911E3C2823006A
:1020700019082000EF0034280C302500BD00803105
:10208000632090310630FB001330FC00AD30FD00C2
:10209000FD0B4828FC0B4828FB0B482800000000DB
:1020A000A530E4008F30E50080319E27903101306B
:1020B0002200A0000030A10000302102031D622890
:1020C0000430200203187E282008F0002108F100C7
:1020D000F035F10D2B30700784000030713D850024
:1020E00000082300E40001310008E50080319E274C
:1020F00090312200A00A0319A10A5C2880317426BD
:1021000090312200EE0188312D26903120302200BE
:10211000EE0088312D26903140302200EE008831CB
:102120002D2690318031742690318831FD259031F3
:1021300091160B178B1705302400920088319726D3
:1021400090314E302200E6000030E70088314A2509
:10215000903101302500AC000130AD0080311126F6
:1021600090310B30FB002630FC005D30FD00FD0B94
:10217000B728FC0BB728FB0BB72800000000803005
:102180002500AC000130AD008031112690310C30BB
:102190002300E4009A30E5008031CD279031C03033
:1021A0002500AC000130AD00803111269031263081
:1021B0002300E4009930E5008031CD279031943040
:1021C0002500AC000130AD00803111269031A830DF
:1021D0002300E4009830E5008031CD279031D430E1
:1021E0002500AC000130AD00803111269031BD30AA
:1021F0002300E4009830E5008031CD279031243071
:10220000FB008330FC00CF30FD00FD0B0529FC0BEB
:102210000529FB0B05298831AE229031D2302300ED
:10222000E4009830E5008031CD27903188313725A2
:1022300090318831DC2390318831FD259031911621
:102240000B178B17003020002A06031D29290130A7
:102250002906031DE92BF5302300E4008F30E5004B
:1022600080319E279031A0302500AC000030AD00B9
:102270008031D6249031803174269031A030E00036
:102280000030E1004730E2000030E30088316F2386
:10229000903170082200A2007108A3007108003C70
:1022A000031D54297008003C031870298831AE22A0
:1022B00090313B302300E4009930E5008031CD2798
:1022C00090313330FB00BB30FC00DF30FD00FD0BF4
:1022D0006729FC0B6729FB0B672900000000010040
:1022E0002300A030E0000030E1003F30E200003089
:1022F000E30088316F23903170082200A20071083A
:10230000A3007108003C031D87297008003C0318D6
:102310009C2920000C120B30FB002630FC005D30A5
:10232000FD00FD0B9129FC0B9129FB0B912900006D
:1023300000008831DC239031A0302300E000003021
:10234000E1003530E2000030E30088316F23903146
:1023500070082200A2007108A3007108003C031D50
:10236000B3297008003C0318B8292000D501D60114
:10237000A0302300E0000030E1003A30E2000030FD
:10238000E30088316F23903170082200A2007108A9
:10239000A3007108003C031DCF297008003C0318FE
:1023A000D62901302000D5000030D600A03023000F
:1023B000E0000030E1002430E2000030E30088312A
:1023C0006F23903170082200A2007108A3007108E9
:1023D000003C031DED297008003C0318E62B8030FB
:1023E0002500AC000130AD00803111269031220073
:1023F00064082500AC00220065082500AD005030BF
:10240000AE009930AF008031612490312200640821
:102410002500AC00220065082500AD008031432571
:10242000903120000C110C121030FB003930FC00F0
:102430000D30FD00FD0B1A2AFC0B1A2AFB0B1A2A81
:102440000000000001302300E40080319E2690311E
:1024500070082000DB007108DC001430F40000304C
:10246000F50080312D2290317008D9007108DA0012
:1024700080302500AC000130AD0080311126903154
:102480002000A201A30159085B07F1005A085C3D36
:10249000F2005C087202031D4F2A5B087102031CE4
:1024A000602A59085B02F1005A085C3BF20072088E
:1024B0005C02031D5D2A71085B02031C602A702AFE
:1024C000220064082500AC00220065082500AD004C
:1024D0006530AE009930AF00803161249031832A9D
:1024E000220064082500AC00220065082500AD002C
:1024F000D030AE009730AF008031612490312000A1
:10250000A20A0319A30A220064082500AC002200D5
:1025100065082500AD008031432590312200640814
:102520002500AC00220065082500AD008031D624CE
:1025300090318031742690310230E40080319E2643
:10254000903170082200EC007108ED006C0820004A
:10255000D70022006D082000D8001430F4000030AD
:10256000F50022006C08F0006D08F10080312D228A
:1025700090317008D9007108DA0008307007F20055
:102580009830713DF30022006D087302031DCA2AC2
:102590006C087202031CDE2A20005908083CF10076
:1025A0005A08031C013E983CF20072085802031DB1
:1025B000DB2A71085702031CDE2AEE2A2200640877
:1025C0002500AC00220065082500AD00E530AE0016
:1025D0009730AF00803161249031012B22006408D4
:1025E0002500AC00220065082500AD000030AE00DB
:1025F0009830AF008031612490312000A20A031985
:10260000A30A220064082500AC002200650825000A
:10261000AD00803143259031220064082500AC00D4
:10262000220065082500AD008031D624903180312C
:102630007426903120005B08F0005C08F1008831BE
:102640005F2290317008E7007108E8007208E90025
:102650007308EA005708F0005808F10088315F223B
:1026600090317008EB007108EC007208ED007308FF
:10267000EE0000302306031D3F2B02302206031D0F
:10268000CC2B6B08F4006C08F5006D08F6006E08A2
:10269000F7006708F0006808F1006908F2006A08AE
:1026A000F3008031AD2390317008E3007108E4003D
:1026B0007208E5007308E60070082300E400710862
:1026C000E5007208E6007308E700A030E80001307A
:1026D000E9000430EA00883100209031EA30E4005B
:1026E0009930E50080319E279031A0302500AC0064
:1026F0000130AD008031D624903180317426903184
:1027000020006308F0006408F1006508F200660824
:10271000F3006308F4006408F5006508F600660835
:10272000F7008031B12590310030F4000030F50021
:102730000030F6007F30F70080314C239031700874
:10274000E3007108E4007208E5007308E600700811
:102750002300E4007108E5007208E6007308E70052
:10276000A030E8000130E9000430EA0088310020A0
:102770009031D930E4009930E50080319E279031C6
:10278000A0302500AC000130AD008031D62490315E
:10279000803174269031D72B23006930E4009730C4
:1027A000E50080319E2790318031742690312000E1
:1027B0000C111F30FB007130FC001E30FD00FD0BC2
:1027C000DF2BFC0BDF2BFB0BDF2B00008831FD2503
:1027D0009031003020005606031DF02B00305506C6
:1027E000031D6F2D8831BF22903103302300E40098
:1027F00080319E26903170082000DD007108DE00D7
:1028000088315F2290317008DF007108E0007208A3
:10281000E1007308E20002302200EE000030EF0019
:102820008831E822903120005F08F4006008F5004C
:102830006108F6006208F7006708F0006808F10018
:102840006908F2006A08F3008031AD239031700806
:102850002200D0007108D1007208D2007308D300A2
:102860007008F4007108F5007208F6007308F700AC
:102870008031B12590310030F4000030F500003097
:10288000F6007F30F70080314C2390317008220031
:10289000D0007108D1007208D2007308D30070080C
:1028A0002300E4007108E5007208E6007308E70001
:1028B000A030E8000130E9000430EA00883100204F
:1028C0009031C830E4009930E50080319E27903186
:1028D000A0302500AC000130AD008031D62490310D
:1028E000803174269031220064082500AC0022005B
:1028F00065082500AD00BB30AE009730AF008031D9
:1029000061249031200063082300E4002000640863
:102910002300E500200065082300E600200066088B
:102920002300E700A030E8000130E9000430EA00AD
:10293000883100209031A030E4000130E50088317A
:102940004022903170082000D9007108DA0014305C
:10295000220064072500AC0000302200653D250000
:10296000AD007008AC027108AD3BA030AE00013084
:10297000AF007008B0007108B10080318625903139
:102980009430AC000130AD0080311126903122002E
:1029900064082500AC00220065082500AD008031E8
:1029A00043259031220064082500AC002200650810
:1029B0002500AD00A630AE009730AF008031612415
:1029C00090310030F0000030F1007A30F2008830B1
:1029D000F30022005008F4005108F5005208F600F8
:1029E0005308F7008031B12590316308F400640882
:1029F000F5006508F6006608F7008031AD239031D8
:102A000070082200D4007108D5007208D60073083F
:102A1000D70070082300E4007108E5007208E600A2
:102A20007308E700A030E8000130E9000130EA0057
:102A3000883100209031A030E4000130E500883179
:102A40004022903170082000D9007108DA0012305D
:102A5000220064072500AC0000302200653D2500FF
:102A6000AD007008AC027108AD3BA030AE00013083
:102A7000AF007008B0007108B10080318625903138
:102A8000220064082500AC00220065082500AD0086
:102A90008031D6249031D4302500AC000130AD0017
:102AA000803111269031220064082500AC002200FC
:102AB00065082500AD0080314325903180317426B2
:102AC00090310B30FB002630FC005D30FD00FD0B2B
:102AD000672DFC0B672DFB0B672D000000000030FD
:102AE00020005606031D762D01305506031D322F9A
:102AF0008831B323903103302300E40080319E26D7
:102B0000903170082000DD007108DE0088315F22FE
:102B100090317008DF007108E0007208E10073086E
:102B2000E20002302200EE000030EF008831E8229F
:102B3000903120005F08F4006008F5006108F6009D
:102B40006208F7006708F0006808F1006908F20001
:102B50006A08F3008031AD23903170082200D00064
:102B60007108D1007208D2007308D3007008F40015
:102B70007108F5007208F6007308F7008031B1257E
:102B800090310030F4000030F5000030F6007F3066
:102B9000F70080314C23903170082200D00071087A
:102BA000D1007208D2007308D30064082500AC007D
:102BB000220065082500AD001530AE009830AF004A
:102BC000803161249031200063082300E40020005C
:102BD00064082300E500200065082300E6002000CB
:102BE00066082300E700A030E8000130E900043067
:102BF000EA00883100209031A030E4000130E50087
:102C000088314022903170082000D9007108DA0024
:102C10001430220064072500AC0000302200653D1E
:102C20002500AD007008AC027108AD3BA030AE00CD
:102C30000130AF007008B0007108B1008031862506
:102C400090319430AC000130AD00803111269031CC
:102C5000220064082500AC00220065082500AD00B4
:102C6000803143259031220050082300E4002200E7
:102C700051082300E500220052082300E60022004C
:102C800053082300E700A030E8000130E9000430D9
:102C9000EA008831002090311D30E4009A30E500D0
:102CA00080319E279031A0302500AC000130AD006E
:102CB0008031D6249031803174269031200067080D
:102CC000F0006808F1006908F2006A08F30067087C
:102CD000F4006808F5006908F6006A08F70080311A
:102CE000B12590317008F4007108F5007208F60003
:102CF0007308F7007B30F0008130F1004F30F200B4
:102D00007930F3008031AD23903170082200CC007F
:102D10007108CD007208CE007308CF000030F400B7
:102D20000030F5007A30F6008830F7008031AD23AE
:102D3000903170082200CC007108CD007208CE00DE
:102D40007308CF0064082500AC0022006508250048
:102D5000AD006930AE009830AF0080316124903111
:102D600022005008F0005108F1005208F200530808
:102D7000F30020006308F4006408F5006508F6001D
:102D80006608F7008031B125903122004C08F4002C
:102D90004D08F5004E08F6004F08F7008031B125C8
:102DA000903170082200C6007108C7007208C80080
:102DB0007308C90070082300E4007108E500720878
:102DC000E6007308E700A030E8000130E9000130B8
:102DD000EA00883100209031A030E4000130E500A5
:102DE00088314022903170082000D9007108DA0043
:102DF0001230220064072500AC0000302200653D3F
:102E00002500AD007008AC027108AD3BA030AE00EB
:102E10000130AF007008B0007108B1008031862524
:102E20009031220064082500AC00220065082500CE
:102E3000AD008031D6249031D4302500AC00013073
:102E4000AD00803111269031220064082500AC00CD
:102E5000220065082500AD00803143259031803186
:102E6000742690312200CA0A0319CB0A0B30FB00EA
:102E70002630FC005D30FD00FD0B3C2FFC0B3C2F91
:0C2E8000FB0B3C2F000000002229452F16
:10347400443084008F3085003530F0000130F10095
:1034840022308600003087008831242698310800D5
:101E000020344434693472346534633474346F3448
:101E10007234793420343A3443343A345C345F34A5
:101E20004D3469346B3472346F3443345C345F3412
:101E30004D3465347334503472346F346A346534DD
:101E4000743473345F344D3469346B3472346F34AA
:101E500043345C345F3431343634463431343834CE
:101E6000343437345F344C3443345F344D34653468
:101E70007434653472345F344C344D34333431341B
:081E800031340D340A34003442
:041E880000340034EE
:0A1E8C0054346534733474340034A8
:041E960000340034E0
:101E9A007A3499348834973400348F3479348F34CF
:041EAA0047349734EE
:0A1EAE0043346134703461340034B1
:0A1EB800533465346C346634003492
:101EC200433461346C3469346234723465340034BE
:0C1ED20052344534533445345434003449
:041EDE000034003498
:041EE2000034003494
:081EE600003400340034003424
:041EEE000034003488
:101EF2002034503472346F346A346534743420348C
:101F02002034203420343A343134363446343134B7
:101F12003834343437345F344C3443344D346534DC
:101F22007434653472345F34423454345F3432343E
:101F32003034313437342E346D3463347034703489
:081F420069340D340A34003447
:101F4A000D340A34203449346E34693474342034FC
:101F5A005334703465346334693461346C346534B1
:101F6A00203455344134523454343A3420345234BF
:101F7A007834203452344234323420346534743460
:101F8A0020345434583420345234423435340D34E5
:041F9A000A340034D1
:101F9E000D340A345034423420346F346E342034CD
:101FAE004C344D3433343134313420343F342034D6
:101FBE003D343E3420345234453453344534543455
:101FCE002034643461346E3473342034313430341C
:0C1FDE007334653463340D340A3400346D
:101FEA00523465346334753420343A34203400343E
:102E8E00203453346F3475347234633465342034E3
:102E9E002034203420343A345F34313436344634DE
:102EAE0031343834343437345F344C3443344D3465
:102EBE0065347434653472345F34423454340D34B2
:042ECE000A3400348E
:102ED20041347434743465346E34743469346F3408
:102EE2006E342C342034543472346F3470342034C1
:102EF20069346E3473347434613462346C346534DE
:0E2F020020342E342E342E340D340A34003494
:102F1000203443346F346D34703469346C3461342C
:102F2000743465347534723420343A3420344D347A
:102F300069346B3472346F344334203437342E3474
:0C2F400030342E3430340A340D340034A8
:102F4C004334583420343A34203420342034203460
:102F5C0020342034203420342034203420342034C5
:0A2F6C002034203470344634003461
:102F760046343134323420343D343A34203420342B
:102F8600203420342034203420342034203420349B
:0A2F960020342034203420340034AD
:102FA0002E342E342E344634313420345334743499
:102FB000613462346C34653420342E34203420344F
:0A2FC0002034203420342034003483
:102FCA0046343234203445346334613472347434D0
:102FDA003E3435342534203449346E3473347434F1
:0A2FEA00613462346C346534003445
:103000002E342E342E344634323420345334743437
:10301000613462346C34653420342E3420342034EE
:0A3020002034203420342034003422
:10302A0046343134323420343D343A342034203476
:10303A0020342034203420342034203420342034E6
:0A304A0020342034203420340034F8
:10305400503472346F3462346C3465346D342034DB
:10306400763461346C3475346534733420344B34C1
:0A30740031342C344B343234003474
:10307E0043346834653463346B3420344F347334E2
:10308E00633469346C346C34613474342E344C349F
:0A309E004D34333431343134003442
:1030A8005234653473346534743420344D344334C5
:1030B80055342034773469346834743469346E3460
:0A30C8002034313430347334003406
:1030D2004C34583420343A342034203420342034D0
:1030E200203420342034203420342034203420343E
:0A30F20020342034753448340034D3
:1030FC004D346F34643465342034533465346C345B
:10310C0066344D3465347434723465342034203470
:0A311C002034203420342034003425
:10312600433461346C3469346234723461347434D7
:1031360069346F346E3420344334433461346C3430
:0A314600203431346E344634003476
:103150002F342F3431346E34463420342B34203421
:103160004334433461346C34203431346E34463467
:0A31700020342034313425340034BB
:10317A005234423436343D34203446347234653461
:10318A0071342E3469346E347034753474342034A6
:0A319A0054344D3452343134003403
:1031A40031343634463431343834343437342034DA
:1031B4004C3443344D3465347434653472342034BF
:0A31C40041344F34503420340034FD
:1031CE004634313420345A34653472346F343D34DD
:1031DE0031346E34663420343A3420342034203482
:0A31EE002034203420343034003443
:1031F8004634333428344D3465347334753472347A
:10320800653429343A3420342034203420342034AE
:0A3218002034203420343034003418
:103222004634323420345334633461346C3465347C
:103232003D3432346E3466343A342034203420340F
:0A32420020342034203430340034EE
:10324C004C3443344D346534743465347234203426
:10325C004C344D3433343134313420343134303413
:0A326C003034753448342034003447
:103276005234453453344534543420344D34433475
:1032860055342034313436344634313438343434D9
:0A3296003734203420342034003493
:1032A00054346534733474342034763461346C347B
:1032B00065347534723473342034463431342034F8
:0A32C0004634323420342034003448
:1032CA0046343134203445346334613472347434CE
:1032DA003E3435342534203449346E3473347434EE
:0A32EA00613462346C346534003442
:1032F400203420342034203420342034203420342A
:103304002034203420342034203420342034203419
:0A331400203420342034203400342B
:10331E004D346F3464346534203443346134703446
:10332E006134633469346D346534743472346534A5
:0A333E002034203420342034003401
:103348004D346F346434653420344334613470341C
:103358006134633469346D3465347434723465347B
:063368000D340A340034AC
:10336E002834463431342F344634323429345E34E2
:10337E00323420342D343134203420343D34203452
:02338E00003409
:103390002834463431342F344634333429345E34BF
:1033A000323420342D343134203420343D34203430
:0233B0000034E7
:1033B2002834463431342F344634323429345E349E
:1033C200323420342D343134203420343D3420340E
:0233D2000034C5
:1033D40052346134703470346F3472347434203441
:1033E400463431342F344634323420343D3420349E
:0233F4000034A3
:1033F6004D346F34643465342034533465346C345E
:1034060066344D3465347434723465340D340A349C
:02341600003480
:10341800563465347234733469346F346E342034FE
:103428003A34203431343734303431343234383467
:0234380000345E
:10343A002834463431342F344634333429345E3414
:10344A00323420342D343134203420343D34203485
:02345A0000343C
:10345C002834463431342F34463432342934203431
:08346C0020343D34203400340B
:020000040001F9
:04000E00E2391316AA
:020000040001F9
:10E00000500049004300310036004600310038001E
:10E0100034003700200038004D0048005A000D0041
:10E020000A004C00430020004D00650074006500AC
:10E03000720020002000200020000D000A000000D7
:10E04000470061006D006D00650020004C0020005D
:10E050003A0020003100750048002000E000200058
:10E060003100300030003000300020006D004800EA
:10E070000D000A00000020002000200020002000E9
:10E08000470061006D006D00650020004300200026
:10E090003A0020003100700046002000E00020001F
:10E0A000310030003000300030006E0046002000AB
:10E0B0000D000A00000020002000200020002000A9
:10E0C0004300610070006100630069006D0065003D
:10E0D0007400720065002000200020002000200055
:10E0E00020002000200020000D000A000000200079
:10E0F0002000200020002000200020002000200020
:10E10000530065006C0066004D00650074007200ED
:10E1100065002000200020002000200020002000BA
:10E1200020002000200020000D000A000000200038
:10E1300020002000200020002000200020002000DF
:10E14000430061006C0069006200720061007400AD
:10E1500069006F006E0020002000200020002000D9
:10E1600020002000200020000D000A0000002000F8
:10E17000200020002000200020002000200020009F
:10E1800054006500730074007300200046003100E5
:10E19000200046003200200046003300200020000E
:10E1A00020002000200020000D000A0000002000B8
:10E1B000200020002000200020002000200000007F
:10E1C000560065007200730069006F006E003A002F
:10E1D00020003100370030003100320038000000EC
:10E1E0007000610075006C0066006A0075006A00CE
:10E1F0006F002000200020002000200020000000F0
:00000001FF
